:10000000B86D0010A5010000A9010000AB010000BF
:10001000AD010000AF010000B10100004288FFEF18
:10002000000000000000000000000000B30100001C
:10003000B501000000000000B7010000B901000098
:10004000BB010000BB010000BB010000BB010000C0
:10005000BB010000BB010000BB010000BB010000B0
:10006000BB010000BB010000BB010000BB010000A0
:10007000BB010000BB010000BB010000BB01000090
:10008000BB010000BB010000BB010000BB01000080
:10009000BB010000BB010000BB010000BB01000070
:1000A00093250000BB010000BB010000BB01000064
:1000B000BB010000BB010000BB010000BB01000050
:1000C000BB010000BB010000BB01000000F002F812
:1000D00000F03EF80AA090E8000C82448344AAF1A4
:1000E0000107DA4501D100F033F8AFF2090EBAE8A2
:1000F0000F0013F0010F18BFFB1A43F0010318475C
:10010000FC5C00001C5D0000103A24BF78C878C178
:10011000FAD8520724BF30C830C144BF04680C600D
:10012000704700000023002400250026103A28BF55
:1001300078C1FBD8520728BF30C148BF0B60704759
:100140001FB59DE8030005F0EAF91FBD10B510BD0D
:1001500005F05CFA1146FFF7F3FF00F01EFB05F017
:100160007AFA03B4FFF7F2FF03BC05F0ABFA000024
:10017000D0F800D0D0F804F070B50023084D0AE0A4
:10018000CE5C04885B1C86EA14269BB235F81660A8
:1001900086EA04240480521E92B2F1D270BD00009F
:1001A0001058000008480047FEE7FEE7FEE7FEE7BC
:1001B000FEE7FEE7FEE7FEE7FEE7FEE70348044949
:1001C000044A054B70470000CD000000B81D001028
:1001D000B86D0010B85D0010B85D0010064802212F
:1001E00041600021016741610B22C260C1630121AE
:1001F0004160002070470000008000402A48002134
:100200000167C160102242618161F122C263274807
:1002100082682748C0E900210846704770B541F25E
:100220008832904215D8642800D290B942F21072F8
:1002300091420ED805290CD31C4CA2681C4B1D689A
:10024000521B5D6805EB4506C6EBC515B2EBC50F45
:1002500001D2002070BD144A0225556040B1154EF0
:10026000B6FBF0F040109061D06155600120506005
:10027000A068C3E90001ECE770B50D4C00250E46FF
:100280006560FFF7CBFF094A06EB46012068C1EB2A
:10029000C61193681B1AB3EBC10FFAD302490220AF
:1002A00048600020656070BD00000940008000408B
:1002B000DC000010001BB700EFF3108010F0010FFE
:1002C00072B64FF080404FF0000202704FF0AA0368
:1002D00003724FF05504047202614FF0FF02426056
:1002E0004FF0030202700372047200D162B6FEE79F
:1002F000704770477047704770477047FFFFFFFFB8
:1003000070B5284C607820B30026274D012810D006
:1003100002280DD1A8686168401A2449884215D383
:100320002348406B400011D5012002F00CF86670A4
:1003300070BDA8686168401A1E498842F8D3002041
:1003400002F001F8A86860600220607026700C203E
:1003500005E020780028EBD1012020700D20BDE8B9
:10036000704001F0E9B8002802D10E490120487020
:10037000704710B501F004FD0A490020487010BD17
:1003800008480121417008498968416070477047F9
:100390007047022803D0032803D100F0AEBD00F05F
:1003A000C9BD70470801001000800040A086010010
:1003B00000C0092040420F0010B591FBF2F491FB00
:1003C000F2F302FB1411C0E9003110BD02F0FF038B
:1003D00043EA032242EA024205F06BB80048704744
:1003E000601D001000210160C0E90110704710205D
:1003F0007047000000487047581D0010C794809A4D
:10040000000000004D0B0000FD4910B5486D0005CF
:100410000CD4FC4A906843F698239468241A9C42B2
:10042000FBD3486D000501D4012010BD052001F06B
:1004300083F8002010BD70B5F24CA668042001F0CE
:100440007BF8F14D03E000BFFFF7DEFF48B1A06885
:10045000801BA842F8D308E0FFF7D6FF08B10120BF
:1004600070BDA068801BA842F6D3002070BD2DE9A6
:10047000F041092001F060F8E44800264FF47A7753
:100480000670C8213846FFF7F7FEDE4CA06842F23E
:100490001075A168091AA942FBD3C8213846FFF795
:1004A000EBFEA068A168091AA942FBD3C82138460F
:1004B000FFF7E2FED648022186708171C670BDE862
:1004C000F0818AB046208DF814004FF000098DF8B5
:1004D000179035208DF81500CE4A31208DF8160082
:1004E0001068CA464FF6FF031840CB4B40F48070AB
:1004F00018431060C948CB49CD4DC0F80090C8489A
:100500000068A0F56C50FF380860C74900F5E0505E
:100510000860C649400A0860F8202870FF2068700B
:10052000A870FFF76BFEBA4CC24A002094F9051080
:1005300052F821102B1803F580530A5C401C83F8F5
:1005400000286028F6D34FF4E175294640F249109F
:10055000FFF792FE294640F29F10FFF78DFE4FF401
:10056000005BDFF8D4825D46207808B1FFF7C8FE53
:10057000A07928B1012818D02078002879D0FCE093
:100580000A2000F0D9FF00F011FE10B1FFF76FFF55
:10059000EAE70120A0715D4684F803A0062000F080
:1005A000CBFF0A2000F0C8FFDEE719222946A24847
:1005B00000F0BCFD98F8180000287CD098F80000E6
:1005C000062873D2DFE800F072030B46464940F27A
:1005D000044000880390D8F80410814266D098F84F
:1005E00009104FF00109404601295FD1D0F80A10E7
:1005F00019B992498969C0F80A100026804617E0A7
:10060000072000F099FFD7F80E00B846871B402F4F
:1006100000D94027A9193A468948193100F086FDCA
:10062000D8F80A003A463044854900F0F3FE3E44CB
:10063000D8F80E004746B042E2D83978012935D1C2
:100640004FF0E0220906C2F88011D7F80A0000F046
:100650000FFF2BE04FF001092BE098F809104FF045
:100660000109032925D16E49764A00260B681360DB
:1006700017E07BE0072000F05FFFD7F80E00871B34
:10068000402F00D94027A9193A466D48193100F08A
:100690004DFD63483A4600688119694800F035FD10
:1006A0003E44D8F80E004746B042E3D898F8180008
:1006B00008B1464600E01CE098F80800C00613D5D3
:1006C0006049012203A8C1F800B005F11801CDF876
:1006D0000CA000F009FD307820B1C8214FF47A70E9
:1006E000FFF7CAFD307E20B1307A800701D5FFF7D1
:1006F000E3FDD8F80E001B3505444F4800F04AFDD5
:1007000030B302204149A0715D4681F800A00B2062
:1007100000F012FFB9F1000F1AD03A484FF000096B
:10072000816842F2107283685B1A9342FBD34FF4E4
:100730002F714FF47A70FFF79FFD3148406D4005EF
:1007400002D50020099001E0099808B9FFF7B4FD2F
:10075000E078401CC0B2E0700C2802D30120A070E9
:1007600014E7A07800283FF413AF0FE701202070B2
:1007700001F028FE012001F0E6FD24480078002861
:10078000F1D0002105A800F021FC0028EBD084F86E
:1007900006A05D4684F803A0E6E61D4C0026FF2077
:1007A0002660A680A671607100F066FF01F012F865
:1007B000FFF714FD00F086FE002000F0BDFE01F002
:1007C00069FFFFF721FEF8B3042000F0B5FE0C4FDF
:1007D000786D0C4D00053AD4FFF72DFEA0B3FFF75E
:1007E0002AFE88B3FFF727FE70B3042000F0A4FEB2
:1007F000A86805497A6D120529D4AA68121A24E05E
:1008000000C009200080004080841E0068000010A5
:10081000BC0000100CED00E00000FA05AC00001078
:10082000B80000109C000010940000109800001008
:1008300035010010600000101C010010505B00002A
:10084000AD1B0010B000001009E08A42D2D3A868A6
:1008500042F21071AA68121A8A42FBD3667100F044
:1008600035FC00F0A3FC80B100F009FE68B1022065
:1008700000F062FE94F90500401C03D10C48806929
:1008800000F0F6FD0120607004E0022000F054FE4C
:1008900066706671FFF7B8FD40B14021054804F06D
:1008A00006FE4022D101034800F02FFCFFF709FEAD
:1008B000505B0000AD1B00102DE9F047FE4A0023FD
:1008C0004FF40077156A4FF4FF79C5F30724DFF87A
:1008D000ECA34FF4E05CDFF8E883FA4E25E0B84281
:1008E00016D213280CD014280CD048450CD0A0F5F3
:1008F0008072FF3A0AD03E2813D81AF8002011E07F
:10090000EAB20FE022460DE055220BE0AA2209E0F0
:10091000604506D208EB0002A2F5805292F8002E44
:1009200000E00022F254401C5B1C8B42D7D3BDE890
:10093000F08770B5E04D2C6B402C00D94024E86A5C
:10094000E96902198A4202D90C1A04216970214608
:10095000FFF7B2FF2246DB49822001F0F0FDE86A92
:100960002044E862286B011BD74829638268A2EB08
:100970000402826005D06978022901D00021017348
:1009800070BD03216970F9E7CF4910B5CF48086001
:100990000D22822001F0D3FDC7490520487010BD0B
:1009A00070B50D46CA49496D490521D4B0F5007F9F
:1009B0001ED3C849C04CB0F5E05F1AD28A68A3695B
:1009C000D21AC54B9A4204D38968A16100216160A3
:1009D0006161BD4900235F39B94A07E0C418144476
:1009E000CE5CA4F580545B1C84F8006EAB42F5D35A
:1009F00070BD626922B98A68A2618A686261A0607A
:100A0000B64A5279002AF3D18A686369D21AB44B84
:100A10009A421CD2B34B01221A708A68A26189687B
:100A20006161A168401A6168884203D9616A88429D
:100A300000D26060062000F07FFD61682A46BDE8B4
:100A40007040A14801F500515F3800F05EBBBDE881
:100A500070400C2000F070BD10B5974CA178E06A92
:100A60004218E1698A4206D9081AA0700520607010
:100A7000022001F01FFDA178E06AFFF791FFA17845
:100A8000E06A0844E062206B421A8F482263836860
:100A9000A3EB0101816002D06178052904D1002116
:100AA0000173BDE810406FE710BD2DE9F041824CA5
:100AB000A178E06A4218E1698A4206D9081AA07052
:100AC00005206070022001F0F5FC7F4D0021A07828
:100AD0007C4B5F3DE26A08E056186F5C9E5DBE424B
:100AE00002D00021A16202E0491C8142F4D3111816
:100AF000E162216B0A1A744922638B68A3EB000040
:100B0000886002D06078052808D1A06A20B1002052
:100B10000873BDE8F04137E70120F9E7BDE8F0814F
:100B2000694810B51F38D0F81110027D09BA21F0BC
:100B3000FF011143604A4902D162C18A49BA4902A0
:100B40001163806888420CD0822001F0B3FC02203F
:100B500001F0B0FC5C4902200873FFF715FF00208C
:100B600010BD012010BD70B55748574D1F380224E5
:100B7000816829B1007B000607D4022001F09AFCAD
:100B80002C73FFF701FF002070BD012070BD10B570
:100B90004D48494C1F388068A178884200D2A07027
:100BA0004949A2785F39822001F0C9FC03206070B6
:100BB0004548A2788168891A81600021017310BDBF
:100BC000414810B51F38816839B1007B000601D556
:100BD000822000E0022001F06DFC3B4900200873F8
:100BE000BDE81040D0E610B5FFF7BDFF00281FD0CC
:100BF000354870215F3802220170002141708270F7
:100C0000C1700171417181710A22C2710172417218
:100C10008172C17230220273012242738173C173E7
:100C200001744174244912208870BDE81040AEE779
:100C300010BD1CB5FFF797FF00286AD02A480A228A
:100C400006210388684600F025FA1F4800225F3815
:100C500080230270437082700121C17020210171D4
:100C600043718271C27141220272542242724F2238
:100C700082724C22C272017341738173C173462226
:100C8000027450234374722383746923C3746E23E4
:100C90000375742343758175C2756C2202766122D7
:100CA0004276732282766822C27601774177817715
:100CB000C1779DF8011019E078000010105B00006A
:100CC00035010010AD1B0010941B0010555342530A
:100CD00000C0092000800040A0860100BC00001078
:100CE00020A10700680000100404000080F8201014
:100CF0009DF8021080F821109DF8031080F8221052
:100D00009DF8041080F82310DE4924208870FFF736
:100D10003EFF1CBD10B5FFF726FF00280CD0DA48B7
:100D200003210170002141708170C170D5490420F8
:100D30008870BDE810402AE710BD10B5FFF713FF1B
:100D4000002810D0D0480021062201704270817026
:100D5000C170017141718171C171CA4908208870E7
:100D6000BDE8104013E710BD10B5FFF7FCFE0028EA
:100D700015D0C44AC448116A491E0B0E03700B0CEF
:100D800043700B0A8370C17000210171417102230D
:100D90008371C17108209070BDE81040F7E610BD66
:100DA00010B5FFF7E0FE002819D0B7480021B54B79
:100DB0000170417081700822C2701A6A140E0471A9
:100DC000140C4471140A8471C271022202724172BD
:100DD0008272C1720C209870BDE81040D7E610BD39
:100DE0002DE9F041A74DA84C0021A8784034A64A2F
:100DF00002E0535C6354491C03468142F9D31F2B24
:100E000072D12068A14988426ED19F4E60685F36DA
:100E10004FF001087060A068B060607B18B9A07BDB
:100E200008B1102802D986F80C8059E0E07B1E2812
:100E3000F9D00FDC12282ED005DC48B30328F2D1FC
:100E4000BDE8F041CFE61528EDD01A28EBD1BDE87A
:100E5000F0415FE702272A2828D010DC23281DD084
:100E600025281ED02828DED1FFF75AFE002826D0DC
:100E7000207B000618D56F70BDE8F04159E52F289A
:100E80001ED05528CFD05A28CDD1BDE8F04154E727
:100E9000BDE8F04194E6BDE8F041CAE6BDE8F041A6
:100EA0007EE7BDE8F0415FE7022016E0FFF738FE7D
:100EB000002804D0207B00060ED485F801802DE6A2
:100EC000FFF72EFE0028FAD0207B000604D485F818
:100ED0000180C5F8288021E6822001F0EBFA377303
:100EE000BDE8F04150E5FFE7822001F0E3FA02207F
:100EF00001F0E0FA0620687010E6624810B541780B
:100F0000022908D003290ED004290FD0052901D1C8
:100F10000021417010BD5C484030C07B2828F9D1C9
:100F2000BDE8104005E5BDE810402DE5822001F048
:100F3000C1FAF8E710B55449022001F0CFFA51493F
:100F40008870487858B101280CD0022001F0B2FA1C
:100F50004D4902205F310873BDE8104014E5BDE83B
:100F600010403DE748484030C07B2A2804D02F2855
:100F700005D1BDE8104098E5BDE810406CE510BD16
:100F8000FFB50246002002EB420501464FF44056F1
:100F90006C4603AA6B1844F82130B34202DD0020EE
:100FA00004B0F0BD3A4F07EB6307DB073F785754B7
:100FB00001D03B095354535C8F0003F00F0353548B
:100FC000BB40491C18440329E4DBE9E7F0B50646B9
:100FD0000020034602462E4C4FF4007700E05B1CD5
:100FE000F55C45B102EB030CA4440CF5805C9CF865
:100FF00000C8AC45F3D0032B3FD302F5C0502044CA
:10100000037F457FC67F03EB0523857F2D0405EB1A
:1010100006652B4451EA03052BD021B919494968CB
:1010200040318B4225D8184B00216C33551825448C
:1010300005F5805595F800585D54491C0C29F5D3E9
:10104000817EC27E01EB0221027D407D120402EB13
:1010500000600C182046FFF793FF40F6F57501E09D
:10106000FFF78EFFC11EA942FAD3A0F57061FF39C8
:1010700001D00020F0BD2046F0BD2032BA42AFD3EF
:10108000F0BD000078000010351B0010555342439E
:1010900035010010FFB5ADA60446E1CE8DE8E100B4
:1010A000022902DA002004B0F0BD6018002100F827
:1010B000011D6946B3FBF2F502FB1535B3FBF2F3F4
:1010C0004D5D00F8015DA042F4D8ECE710B504F0E6
:1010D0008CF804F076F8A1494FF40052C1E90020E1
:1010E000A0F5F420886010BDF8B514469B4E0A4662
:1010F0000B19716800258B4200D90A1B0346009426
:10110000306804F0C0F82846F8BDF8B51446934E90
:101110000A460B19716800258B4200D90A1B034649
:101120000094306804F0AFF82846F8BD10B50B46BF
:1011300001460024184604F07BF8204610BD2DE936
:10114000FC410746002090460E46ADF800000446DC
:101150000EE0351B402D00D9402539192A4680481C
:10116000FFF7E4FFAAB27E496846FFF705F82C4472
:10117000B442EED33919424601A8FFF7D7FFBDF8B4
:101180000000BDF80410884202D10120BDE8FC81B6
:101190000020FBE70021425C12B9491C1829FAD350
:1011A000182901D000207047012070472DE9F04137
:1011B0006A4C00270C3488B0A770E770DFF8A48170
:1011C0004FF40056277101251922314601A8FFF777
:1011D000ADFF022216213046FFF7B1FF00287DD077
:1011E000DDF81210022206F11900FFF7A8FF00280F
:1011F00074D09DF80400062829D2DFE800F0290306
:101200000329291CD8F87410DDF80E30491C8B42D4
:101210001DD2D8F87420DDF80E30D21ADDF8123065
:10122000521C9A4213D3DDF80E20DDF812301A4416
:101230008A420CD80CE0DDF81210B1F5F42F00D979
:10124000A570DDF81610C1F30B41102900D0A57070
:10125000012803D0022801D0052839D1022206F244
:101260001D4168460097FFF761FF0099029889B217
:10127000884200D0A570012206F2254168460097F9
:10128000FFF754FF0099BDF80500C9B2884200D0AD
:10129000A5709DF8040002281AD1042206F24941E3
:1012A00068460097FFF742FFDDF816000099884274
:1012B00000D0A570012206F24D4168460097FFF765
:1012C00035FF00989DF80710C0B2814200D0A5708C
:1012D0009DF81C00401EFE2802D200E01EE0A57012
:1012E000BDF80500A0F57F41FF3901D0432802D1A8
:1012F0009DF8070020B901A8FFF74CFF00B9A570C1
:10130000DDF812001B36064401A8FFF743FF30B199
:10131000E07880B1217988420DD012E0A5709DF867
:101320001C0010B92079401C2071E078401CC0B22C
:10133000E0700C2801D3A57003E0A07800283FF4EA
:1013400043AFA07808B0BDE8F081000030313233FF
:10135000343536373839414243444546B0000010F1
:10136000AD1B0010C85B00004F4A104710B572B6A5
:1013700033244E4B10C307C34D484FF47A710068B5
:10138000B0FBF1F01860191D4848FFF7EDFF62B699
:1013900010BD464A32231360C2E9010144484FF4AC
:1013A0007A710068B0FBF1F0D06002F114011046D0
:1013B000DAE73E4A34231360C2E901013C484FF4A6
:1013C0007A710068B0FBF1F0D06002F114011046B0
:1013D000CAE710B572B60624364900BF51F824207A
:1013E000824212D93349783951F82410814207D109
:1013F00021460846FFF7CDFF21460846FFF7D9FFF3
:1014000021460846FFF7C5FF02E0641C1D2CE5D904
:1014100062B610BD2DE9F041274C236803B9206066
:10142000224D00202835636803E00F5C1E18401C25
:10143000AF559042F9D398184FF480766060B0426F
:1014400013D12068FFF7C5FF184D1435286800B187
:10145000FEE71649324628312068FFF787FF2868E3
:1014600000B1FEE70020606020600020BDE8F08150
:1014700072B61249124A01401160FEF779BE46F277
:10148000044000210088A0F51942993A0AD04FF48F
:10149000C0404FF4002208C890421944FBD309B160
:1014A0000020704701207047F11FFF1FF01B001044
:1014B000D8000010C85B0000C400001080FFFF1FB0
:1014C00008ED00E0002070476949C20702D04FF4E0
:1014D00080028A61800702D54FF4001088610020E5
:1014E00070476349C20702D04FF48002CA61800787
:1014F00002D54FF40010C86100207047014600205B
:101500005B4ACB0703D053695B0200D501208907F2
:1015100004D55169890201D540F00200704710B529
:101520000446FFF7EBFF0346FFF7DBFF24EA030067
:10153000FFF7CAFF002010BD70B54E4B50B159687F
:10154000042403250226052907D2DFE801F0072B32
:101550004A718E0000205860986070BD042807D042
:10156000052809D0012402287AD0012808D00FE0EC
:101570000320FFF7B6FF46E0BDE870400120B0E76A
:101580000320FFF7AEFF0BE0FFF79EFF5C6070BD2E
:101590000E28FCD10320FFF7A4FF0220FFF794FFE1
:1015A0000120F1E706280AD0032810D00A2813D01A
:1015B000092811D00D280FD00C28D9D070BD0320D8
:1015C000FFF78FFF0220FFF77FFF5E6070BD0320F3
:1015D000FFF787FF012027E00320FFF782FF0220AB
:1015E00012E0062813D00A281AD00928C8D00C28DF
:1015F000BED00D28F0D00F28E8D10320FFF771FFEF
:101600000220FFF761FF0120BDE870405CE79868A9
:1016100010F01F0F00F101009860D7D102201BE0ED
:101620000320FFF75EFF0220FFF74EFF5D6070BDF5
:10163000072806D00A289BD00B2811D009289FD054
:1016400070BD0220FFF74DFF986810F03F0F00F1CA
:1016500001009860F4D10120BDE870405FE7FFE72A
:101660000320FFF73EFF02208EE70628A7D08FE772
:1016700000C00920CC0000104F4810B52021C0F850
:10168000A01100BFD0F8A0114906FBD50521C0F874
:1016900004114FF04472C0F8A8214FF48062C0F8E2
:1016A000AC210122C0F80C210B23C0F88430C0F813
:1016B0008020AA22C0F88C205523C0F88C3000BFAF
:1016C000D0F888406401FBD50324C0F88040C0F8FE
:1016D0008C20C0F88C30C0F808113849C0F8C4100C
:1016E0000021C0F8C811D0F888106FEA11618A078C
:1016F0003349D0F80C2102F0030207D07AB3012A53
:1017000044D0022A47D0032A4ED13AE02AB1012A16
:1017100013D0022A24D0032A46D1D0F88820D0F84A
:101720000431C2F30742DBB2521C5B1C5A43D0F8AF
:101730008830244CC3F30E030EE0D0F88820D0F894
:101740000431C2F30742DBB2521C5B1C5A43D0F88F
:1017500088301D4CC3F30E035B1C634321E010E093
:10176000D0F88820D0F80431C2F30742DBB2521C13
:101770005B1C5A43D0F888304FF47A44C3F30E030D
:10178000EAE7D0F80421114BD2B209E0D0F80421E5
:101790000F4BD2B204E0D0F804214FF4FA43D2B296
:1017A000521CB3FBF2F20A60016821F4704141F46B
:1017B0000051016010BD000000C00F40DC96688140
:1017C000D800001000127A0000366E0100093D00BA
:1017D000001BB700F0B5FF4800218162016821F4C9
:1017E00040310160016C21F4403141F40031016469
:1017F000F9498215CA610B6843F480730B60036872
:1018000023F440530360036C23F4405343F4005328
:1018100003644024CC610B6843F040030B60036811
:1018200023F440630360036C23F4406343F40063D8
:1018300003642023CB610B6843F020030B60036833
:1018400023F440730360036C23F4407343F4007388
:1018500003641023CB610D6845F010050D60C56869
:1018600025F00C05C560C56C25F00C0545F0080594
:10187000C5645502CD630E6A46F400360E620669F1
:1018800026F440560661066D26F4405646F400568E
:1018900006658C650C6C44F040040C64046924F00B
:1018A0000304641C0461046D44F0030404650469CA
:1018B00024F00C04241D0461046D44F00C04046540
:1018C000046924F0300444F010040461046D44F011
:1018D00030040465046924F0C00444F04004046149
:1018E000046D44F0C0040465046924F4407444F4B5
:1018F00080740461046D44F440740465046924F444
:10190000406444F480640461046D44F440640465FC
:10191000046824F4404444F400440460046C24F457
:1019200040440464046824F4402444F40024046023
:10193000046C24F440240464446824F00C044460DF
:10194000446C24F00C044464CD610C6824F400342D
:101950000C60446824F030044460446C24F030048B
:1019600044F0200444649402CC610D6825F4802581
:101970000D60C56845F44025C560C56C25F440255B
:1019800045F40025C564C56845F04045C560C56C93
:1019900025F0404545F00045C564056825F0300553
:1019A00045F010050560056C25F0300545F0200573
:1019B0000564056825F0C00545F040050560056C27
:1019C00025F0C0050564056925F0406545F0806592
:1019D0000561056D25F040650565056825F0404504
:1019E00045F080450560056C25F0404545F0004513
:1019F0000564456825F003056D1C4560456C25F0C0
:101A000003054564056825F4401545F48015056017
:101A1000056C25F4401545F400150564056825F4AA
:101A2000400545F480050560056C25F44005056416
:101A3000C56845F44035C560C56C25F4403545F4AE
:101A40000035C564C56845F44045C560C56C25F4DE
:101A5000404545F40045C564C56845F44075C5601A
:101A6000C56C25F4407545F40075C564C56825F45A
:101A70004055C560C56C25F44055C56495038D631C
:101A80000E6A46F480060E62C66826F44066C6609A
:101A9000C66C26F44066C66456038E630F6A47F42C
:101AA00000170F62C76827F44017C760C76C27F498
:101AB0004017C76497048F630F6A47F080670F620F
:101AC000C76827F03007C760C76C27F03007C764C6
:101AD0008C630C6A44F480240C62446824F04074E3
:101AE00044F080744460446C24F04074446444685E
:101AF00024F4400444F480044460446C24F440041E
:101B00004464046844F00C040460046C24F00C0485
:101B10000464046844F003040460046C24F00304C7
:101B20000464446824F0406444F080644460446C7D
:101B300024F0406444F000644464446824F0405459
:101B400044F080544460446C24F0405444F0005409
:101B50004464C46824F0405444F00054C460C46C2D
:101B600044F04054C464C46924F44024C461C46D86
:101B700044F44024C4655404CC670C6E44F00074F3
:101B80000C66446824F4401444F480144460446CAB
:101B900024F4401444F400144464446824F440449D
:101BA00044F480444460446C24F4404444F40044CD
:101BB0004464446824F4402444F480244460446C25
:101BC00024F4402444F400244464446824F440345D
:101BD00004E0000000C0024000C0092044F480344A
:101BE0004460446C24F4403444F400344464446855
:101BF00024F440544460446C24F4405444F40054AD
:101C00004464CD610C6844F480040C60446824F49E
:101C100040644460446C24F4406444F400644464CC
:101C2000CE610C6844F400140C60446A24F04074E3
:101C300044F000744462446E24F0407444F0007434
:101C40004466446A24F0406444F000644462446E94
:101C500024F0406444F000644466846824F00C047A
:101C60008460846C24F00C0444F00804846402242E
:101C7000CC630C6A44F002040C62846824F0030410
:101C80008460846C24F0030484640124CC630C6AB3
:101C900024F001040C62C46824F00304C460C46C22
:101CA00024F00304A41CC4641402CC630C6A44F43E
:101CB00080340C62046924F440040461046D24F44B
:101CC00040040465C414CC650C6C24F400640C64FA
:101CD000046924F440140461046D24F44014046580
:101CE0000415CC650C6C24F480640C64C46824F482
:101CF000400444F48004C460C46C24F4400444F4FC
:101D00000004C464C46824F0C004C460C46C24F03B
:101D1000C00444F08004C464D402CC630D6A45F46A
:101D200000250D62C56825F0C005C560C56C25F0AD
:101D3000C00545F08005C564CC630C6A44F40024FA
:101D40000C62846824F440748460846C24F44074CD
:101D500044F400748464CB630B6A43F010030B6299
:101D6000836823F440338360836C23F4403343F46B
:101D7000003383648A63086A40F480700862F0BDAF
:101D8000FA4800214FF00112818001704170C0E9D2
:101D900002217047F5491C31002000F09FBB10B5AF
:101DA000F24C1434A288402A00D9402280202168B5
:101DB00000F0C5FB216801442160A188081AA080B9
:101DC00010BD10B5E94C00201434216800F086FBEA
:101DD000216801442160A188081AA08010BD00225A
:101DE0001146802000F0ABBBE149002000F076BB3B
:101DF00070B5DE48DD4D1C3005F11405007810F09B
:101E00001F040AD0D949DA4B01F11C004A78007945
:101E1000012C06D0022C26D109E0D448001D2860F0
:101E20001DE002B3897888421DD2002015E000F041
:101E30008F04200605D504F00F064FF48030B04023
:101E400001E00120A0400AB922070CD18A680242B1
:101E500009D0C9680142E8D0012018802B60FFF743
:101E60009EFF012070BD002070BD024670B5BF48C6
:101E7000BE4C1C30017811F01F030146498804D084
:101E8000012B29D0022B27D111E0012924D132B115
:101E9000012000F0BDFAA08840F0020005E000201B
:101EA00000F0B6FAA08820F00200A08021E00079BE
:101EB00000F08F00030605D500F00F034FF48035C6
:101EC0009D4001E00125854063782BB1030703D0D5
:101ED000A3682B4200D009B1002070BD22B100F0F0
:101EE000E9FAE068284303E000F0EEFAE068A8436E
:101EF000E060012070BD9D4810B51C30007810F0E6
:101F00001F0F9A4800F11C00C0782AD1974914315C
:101F1000012807D001F108020228937806D003288F
:101F20001FD112E093480860122012E0924800226C
:101F300004E004780CB144882044521C9342F8D148
:101F4000027872B10860408803E08C481844086049
:101F500000788A88824200D98880FFF720FF01201C
:101F600010BD002010BD2DE9F84F804F00201C3718
:101F70000090B8787D4E4FF000094FF0010A4FF401
:101F8000803B00286BD07C4C65E06078022804D050
:101F9000042841D005285CD141E06179B8788142BC
:101FA00038D170702079B0707049002011F11001A3
:101FB00001F80090401C0428FAD301254FEA0608D6
:101FC0000AFA05F0D8F80810084202D0284600F0B6
:101FD0005DFAD8F808100BFA05F0084203D045F076
:101FE000800000F053FA6D1C102DE9D34FF0011062
:101FF000C8E90209012000F00CFAE0794006B8F8BF
:10200000040002D540F0010001E020F00100A8F832
:1020100004001EE060881DE0E078009019E0009860
:10202000B8B9A07800F08F05280604D505F00F0197
:102030000BFA01F001E00AFA05F0B168014320460D
:10204000B16000F0FCF9284600F016FA284600F0CE
:1020500027FA207804442078002896D11FE086F8DB
:10206000019001245546D846B16805FA04F00842AB
:1020700002D0204600F00AFAB16808FA04F00842DB
:1020800003D044F0800000F001FA641C102CEBD364
:102090004FF00110C6E90209002000F0BAF9B87843
:1020A0007178884202D10120BDE8F88F0020FBE75B
:1020B0002DE9FC5F2D4D00273E466878BB46B846AB
:1020C000002871D0BA462C4C05F11C0968E06078F4
:1020D000022804D0042808D005285FD119E06079CF
:1020E000697888425AD0608859E0A77899F8041036
:1020F000E6784FF00008B94250D199F80200B0429A
:102100004CD11A484FF0010A103010F807B0C655EC
:1021100044E099F80410B94240D1A17801F08F0150
:102120000191090605D5019901F00F024FF48031A4
:1021300001E0019A01219140009199F80200B0421A
:102140001ED1A8680843A860E9680098814320462A
:10215000E96000F074F9019800F08EF9019800F040
:102160009FF9009948EA010818E00000E400001017
:10217000181D0010405C0000525C0000735C000001
:102180005E450BD118EA010F08D1A8688843A86002
:10219000E8688843E860019800F078F92078044402
:1021A0002078002893D15046BDE8FC9F2DE9F041EE
:1021B000494C0027A4F108062178A4F11C05082841
:1021C00063D2DFE800F06204647262628381FFF729
:1021D000E1FD2078C00900F04EF9E088B080207859
:1021E000C0F34111F1BB61780C294AD2DFE801F05C
:1021F0000609490B49101A1D1F253142FFF7F8FD4A
:102200004DE0002000E00120FFF72FFE50B306E074
:1022100010F01F0F35D1A07840F080002870BDE885
:10222000F041DCE5FFF767FE39E000202AE010F01E
:102230001F0F26D128481B381AE010F01F0F20D19D
:10224000FFF791FE70B1FFF7CAFDBDE8F041FEF760
:102250009FB800F01F00012813D1687810B12079D1
:10226000A97800E00DE088420BD21B490C390844E4
:1022700030601CE000F01F00012802D1FFF718FFBA
:10228000C4E7802000F016F9B780BDE8F0810806A9
:1022900008D4B0880028F8D0FFF793FDB088002854
:1022A000EFD0F2E7BDE8F0419EE5080602D5BDE8B3
:1022B000F04174E528780106E7D500F07F0028702A
:1022C000BDE8F04100F054B8802000E00020BDE8F7
:1022D000F04100F0F9B800000001001001460007CD
:1022E000C00E090600D5401C7047DA491022C1F81B
:1022F0000822C1F8100200BFD1F80002C006FBD5C9
:102300007047D44A1023C2F80832C2F8100200BF46
:10231000D2F80002C006FBD5C2F80832C2F810128B
:10232000D2F80002C006FBD57047CA493022C1F876
:102330000822C1F8100200BFD1F800028006FBD5C8
:10234000D1F81402704710B5040001D0012000E05C
:1023500000204FF4807141EA0041BF48FFF7D1FFF0
:10236000BE494FF000700CB1886710BDC86710BD42
:1023700030B5BB49BB4D41EA004421462846FFF732
:10238000C0FF21462846BDE83040BAE7B1480021E9
:10239000C0F848124021C0F84C120122C0F848226F
:1023A000C0F84C12D0F80012C905FBD54FF0FF3130
:1023B000C0F83812C0F83412C0F808120C21C0F866
:1023C00004127047A84800B5C16821F0405141F09F
:1023D0000051C160C16C41F04051C164A3491A2051
:1023E0000860091D0A6830EA0202FBD14FF0E021C3
:1023F0004FF08070C1F880029D4B202283F80024AA
:10240000C1F80001FFF7C2FF00205DF804EBAFE761
:10241000704710B500B101204FF4807444EA0041C8
:102420009448FFF76EFF8B480321C0F8441200BFA9
:10243000D0F80012C905FBD5C0F8084210BD10B590
:1024400002468078FFF74AFF8249D1F844320124DE
:1024500084402343C1F84432C1F848029088C1F84F
:102460004C0200BFD1F80002C005FBD54FF48070CC
:10247000C1F8080210BD704700B5FFF72FFF7E4975
:102480005DF804EB41EA004089133AE700B5FFF735
:1024900025FF79495DF804EB41EA0040774930E7D0
:1024A00000B5FFF71BFF74495DF804EB41EA0040FB
:1024B000891326E700B5FFF711FF6F495DF804EBBC
:1024C00041EA00406E491CE700B5FFF707FF6A4983
:1024D0005DF804EB41EA0040891312E700F00F02B7
:1024E000012370B503EB82035A4AC2F8283200BFB9
:1024F000D2F820321C05FBD5C3F309030024DD1CF0
:1025000005E000BFD2F8186241F8046B641CB4EB1C
:10251000950FF7D30021C2F8281241F24821C1409B
:10252000C9070AD1FFF7DAFE4FF4A06141EA004083
:10253000FFF7DBFE5348FFF7D8FE184670BD70B5B5
:1025400013460546434C00F00F00022202EB8000C8
:10255000C4F82802C4F824320020DA1C05E000BFC9
:1025600051F8046BC4F81C62401CB0EB920FF7D317
:102570000020C4F828022846FFF7B0FE4FF4A061FF
:1025800041EA0040FFF7B1FE3F48FFF7AEFE1846B4
:1025900070BD2DE9F0412F4DD5F80032C5F8083255
:1025A000180721D52C48FFF7A0FE3848FFF7BDFEDD
:1025B000C10605D5FFF7EAFEBDE8F041FDF7D9BE3B
:1025C000810705D5BDE8F04100F00100FDF7CBBE65
:1025D000010709D5400703D5BDE8F041FDF7D0BE9E
:1025E000BDE8F041FDF7D3BE294E58074FF0010773
:1025F0001CD4BDE8F0810024D5F8302207FA04F19C
:102600000A4210D06008C5F8381200BFD5F8001291
:102610008906FBD5D5F81412E2070CD056F8201025
:1026200009B103208847641C202CE5D3D5F830027B
:102630000028E0D1DDE73CB9490705D5316819B17B
:10264000012088470124D7E756F820100029EAD056
:102650000220E7E700C000500005FE0000C009208E
:10266000000180000005D00000C00240F4CF0050FF
:1026700018E000E00005D80000054000000120003F
:10268000000101000005F2000005FA000002FE0052
:10269000E45C000019480621016107210160002166
:1026A0004161416202214160C168C906FCD400E079
:1026B0008168C1684907FBD4002070470F498860D2
:1026C000C868C006FCD48868704700B50B4602464F
:1026D00004E000BF12F8010BFFF7F0FF5B1EF9D218
:1026E00000BD00B50B46024604E00020FFF7E6FF00
:1026F00002F8010B5B1EF8D200BD0000008008400C
:102700002DE9F047F74E80464FF080773068BC11D6
:10271000F54DB84249D100BF00BF00BF00BF00BFA8
:1027200000BF00BF00BF00BF00BF00BF00BF00BFB1
:1027300000BF00BF00BF00BF00BF00BF00BF00BFA1
:1027400000BF00BF00BF00BF00BF00BF00BF00BF91
:1027500000BF00BF00BFEC631520FFF7AFFF0020F4
:10276000FFF7ACFF00F0FF09AC6300BF00BF00BF84
:1027700000BF00BF00BF00BF00BF00BF00BF00BF61
:1027800000BF00BF00BF00BF00BF00BF00BF00BF51
:1027900000BF00BF00BF00BF00BF00BF00BF00BF41
:1027A00000BF00BF00BF00BF00BF00BF00BF00BF31
:1027B00000BF00BF00BF00BF00BF00BF00BF00BF21
:1027C00000BF00BF00BF00BF00BF00BF00BF00BF11
:1027D00000BF00BF00BF00BF00BF00BF00BF00BF01
:1027E00000BF00BF00BF00BF00BFEC630620FFF7C3
:1027F00065FFAC6300BF00BF00BF00BF00BF00BFEC
:1028000000BF00BF00BF00BF00BF00BF00BF00BFD0
:1028100000BF00BF00BF00BF00BF00BF00BF00BFC0
:1028200000BF00BF00BF00BF00BF00BF00BF00BFB0
:1028300000BF00BF00BF00BF00BF00BF00BF00BFA0
:1028400000BF00BF00BF00BF00BF00BF00BF00BF90
:1028500000BF00BF00BF00BF00BF00BF00BF00BF80
:1028600000BF00BF00BF00BF00BF00BF00BF00BF70
:1028700000BF00BFEC630120FFF720FF4FEA880094
:10288000FFF71CFF3068B84202D14846FFF716FF39
:10289000AC6300BF00BF00BF00BF00BF00BF00BFF0
:1028A00000BF00BF00BF00BF00BF00BF00BF00BF30
:1028B00000BF00BF00BF00BF00BF00BF00BF00BF20
:1028C00000BF00BF00BF00BF00BF00BF00BF00BF10
:1028D00000BFBDE8F0872DE9FC5F8846044601A9EA
:1028E000824800F05DFB824D824E834FF0BB032097
:1028F0008DF8000020098DF8010020018DF80200FC
:102900004FF000098DF8039000BF00BF00BF00BF6B
:1029100000BF00BF00BF00BF00BF00BF00BF00BFBF
:1029200000BF00BF00BF00BF00BF00BF00BF00BFAF
:1029300000BF00BF00BF00BF00BF00BF00BF00BF9F
:1029400000BF00BF00BF00BFDFF89CB14FF4802A7A
:10295000CBF83CA004216846FFF7B7FE0024002016
:10296000FFF7ACFEC0B28DF8040000E003E018F8F9
:102970000410884208D082202860222030607846E7
:1029800038608220BDE8FC9F641CB4F5805FE6D30C
:10299000CBF838A000BF00BF00BF00BF00BF00BF22
:1029A00000BF00BF00BF00BF00BF00BF00BF00BF2F
:1029B00000BF00BF00BF00BF00BF00BF00BF00BF1F
:1029C00000BF00BF00BF00BF00BF00BF00BF00BF0F
:1029D00000BF00BFC5F800907846C6F80090386088
:1029E0000020CFE72DE9F0474FF0000900BF00BFFE
:1029F00000BF00BF00BF00BF00BF00BF00BF00BFDF
:102A000000BF00BF00BF00BF00BF00BF00BF00BFCE
:102A100000BF00BF00BF00BF00BF00BF00BF00BFBE
:102A200000BF00BF00BF00BF00BF00BF2E4E4FF46D
:102A30008025F5639F20FFF741FE0020FFF73EFE53
:102A400000F0FF080020FFF739FEC4B20020FFF7B6
:102A500035FEC1B2B56300BF00BF00BF00BF00BFFD
:102A600000BF00BF00BF00BF00BF00BF00BF00BF6E
:102A700000BF00BF00BF00BF00BF00BF00BF00BF5E
:102A800000BF00BF00BF00BF00BF00BF00BF00BF4E
:102A900000BF00BF00BF164D164E174FB8F1C20F52
:102AA00001D1202C07D08220286021203060784678
:102AB000386082200DE70B4814291FD0152920D03B
:102AC000162922D0182923D0C0F800900020FFF743
:102AD00017FEC5F800907846C6F8009038600020D0
:102AE000F7E600001001001000C00920A0860100D8
:102AF0006C00001070000010740000104FF4801182
:102B000001E04FF400110160E0E74FF48001FAE7C3
:102B10004FF08071F7E72DE9F34FC3B080460024F2
:102B20004FF0820AFE4DFF4EFF4F4FF0210BA146A2
:102B300041A9FE4800F034FA00286CD100F09CFA5C
:102B400002208DF800004FEA18108DF8010004EB08
:102B500008108DF8020044988DF8039000EB0421D2
:102B60004FF4807201A802F02BFC00BF00BF00BF31
:102B700000BF00BF00BF00BF00BF00BF00BF00BF5D
:102B800000BF00BF00BF00BF00BF00BF00BF00BF4D
:102B900000BF00BF00BF00BF00BF00BF00BF00BF3D
:102BA00000BF00BF00BF00BF00BFE1494FF480205D
:102BB000C8634FF482716846FFF787FDDC494FF424
:102BC0008020886300BF00BF00BF00BF00BF00BF00
:102BD00000BF00BF00BF00BF00BF00BF00BF00BFFD
:102BE00000BF00BF00BF00BF00BF00BF00BF00BFED
:102BF00000BF00BF00BF00BF00BF00BF00BF00BFDD
:102C000000BF00BF641CE4B2102C91D341A9C74897
:102C100000F0C6F948B1C5F800A07846C6F800B083
:102C20003860822045B0BDE8F08F00F06FFAC5F83B
:102C300000907846C6F8009038600020F2E72DE951
:102C4000F04F89B0DFF8D8825FEA020B4FF0000640
:102C500007910FD04FF4805501462A466846FDF78C
:102C6000ABFBDDE90047284602F054FB5FEA0009B0
:102C70000CD016E08621AB48C8F80010092101608D
:102C80007946A9480160862009B0CCE78221A54891
:102C9000C8F80010222101607946A3480160822013
:102CA000F2E7ABEB0605C7F580504FF0000AA842EB
:102CB00000D20546B5F5805F04D02046494600F0B5
:102CC000A3FCD8B907982A46811907EB090002F03E
:102CD00077FB204600F01DFC80B920464946FFF7EF
:102CE0001AFF58B920464946FFF7F5FD78B10AF1B9
:102CF000010000F0FF0ABAF1030F05D3484602F0C5
:102D000038FBD8F80000BFE7BAF1000FE1D12E443C
:102D10000027641C5E45C4D3484602F02AFB814963
:102D20000020C8F80000086079467F480160002054
:102D3000AAE72DE9FF4F8DB00D46DDF8689000261B
:102D4000774C07935FEA09013FD04FF48057014663
:102D50003A466846FDF730FBDDE900B10C913A4692
:102D6000691C6846FDF728FBDDE90010CDE9040188
:102D70003A4668460F99FDF71FFBDDE9008500BF65
:102D8000A9EB0607C5F58050B84200D2074625B129
:102D9000D8457CD10C98854279D14FF4805002F00F
:102DA000B9FA5FEA000A1BD0D8454FD10C9885428A
:102DB0004CD12A464FEA0830514600F0FEFA000690
:102DC00018D5504602F0D5FA79E0862020605548A3
:102DD00009210160784654490860862011B022E735
:102DE000822020604F482221016079464E480160D0
:102DF0008220F3E70598804509D1049901EB003062
:102E0000C1F58052514400F0D8FA0006D9D44046AA
:102E100000F07FFB0006D4D407983A46811905EBF1
:102E20000A0002F0CDFAEA194FEA0830514601F0E3
:102E3000DCF90006C5D40599884533D1049800EB28
:102E400001300499C1F58052514427E00599884525
:102E50000AD1049800EB01300499C1F58052514623
:102E600000F0ABFA0006ACD4404600F052FB00067E
:102E7000A7D407983A4681190F98304401F0B5F964
:102E800000069ED4059988450CD1049800E00DE019
:102E900000EB01300499C1F58052514601F0A5F9CB
:102EA00000068ED4504602F064FA0AE007983A46CB
:102EB00081190F98304401F098F9000601D5206877
:102EC0008CE73E44002508F101084E45FFF458AF59
:102ED00014490020206008607846134908600020EB
:102EE0007CE71448006870474FF4805070472DE924
:102EF000F04FDFF82C80DFF82CB089B00F000446CB
:102F00004FF0000633D04FF4805501462A466846FC
:102F1000FDF752FADDE900A105912A4621460BE0B2
:102F20006C0000107000001074000010A0860100FA
:102F300000C009201001001006A8FDF73DFADDE9E8
:102F400006404FF00009BD1BC0F58051A94200D2D8
:102F50000D4620B1544515D10599884212D120461D
:102F600000F0D7FA00060DD5D8F800008CE68621CF
:102F7000C8F800100921CBF8001079463B480160E1
:102F8000862081E62E44641C4846BE42DBD3C8F846
:102F900000007946CBF8000034480160002073E659
:102FA0002DE9F041324C0F460646A56806E0A068C0
:102FB000401BB04202D30120BDE8F081384600F04A
:102FC00003F80028F3D1F7E770B5044600BF00BF4F
:102FD00000BF00BF00BF00BF00BF00BF00BF00BFF9
:102FE00000BF00BF00BF00BF00BF00BF00BF00BFE9
:102FF00000BF00BF00BF00BF00BF00BF00BF00BFD9
:1030000000BF00BF00BF00BF00BF00BF194E4FF49C
:103010008025F5630520FFF751FB0020FFF74EFBED
:103020002070B56300BF00BF00BF00BF00BF00BF7E
:1030300000BF00BF00BF00BF00BF00BF00BF00BF98
:1030400000BF00BF00BF00BF00BF00BF00BF00BF88
:1030500000BF00BF00BF00BF00BF00BF00BF00BF78
:1030600000BF00BF207800F0010070BD74000010A8
:103070000080004000C0092070B500BF00BF00BF45
:1030800000BF00BF00BF00BF00BF00BF00BF00BF48
:1030900000BF00BF00BF00BF00BF00BF00BF00BF38
:1030A00000BF00BF00BF00BF00BF00BF00BF00BF28
:1030B00000BF00BF00BF00BF00BFFE4C4FF4802523
:1030C000E5630620FFF7FAFAA56300BF00BF00BF63
:1030D00000BF00BF00BF00BF00BF00BF00BF00BFF8
:1030E00000BF00BF00BF00BF00BF00BF00BF00BFE8
:1030F00000BF00BF00BF00BF00BF00BF00BF00BFD8
:1031000000BF00BF00BF00BF00BF70BD70B500BFF3
:1031100000BF00BF00BF00BF00BF00BF00BF00BFB7
:1031200000BF00BF00BF00BF00BF00BF00BF00BFA7
:1031300000BF00BF00BF00BF00BF00BF00BF00BF97
:1031400000BF00BF00BF00BF00BF00BF00BFD94C21
:103150004FF48025E5630420FFF7B0FAA56300BFB4
:1031600000BF00BF00BF00BF00BF00BF00BF00BF67
:1031700000BF00BF00BF00BF00BF00BF00BF00BF57
:1031800000BF00BF00BF00BF00BF00BF00BF00BF47
:1031900000BF00BF00BF00BF00BF00BF00BF70BDC9
:1031A00070B5064600BF00BF00BF00BF00BF00BF34
:1031B00000BF00BF00BF00BF00BF00BF00BF00BF17
:1031C00000BF00BF00BF00BF00BF00BF00BF00BF07
:1031D00000BF00BF00BF00BF00BF00BF00BF00BFF7
:1031E00000BF00BFB34D4FF48024EC635020FFF7C5
:1031F00065FAAC6300BF00BF00BF00BF00BF00BFE7
:1032000000BF00BF00BF00BF00BF00BF00BF00BFC6
:1032100000BF00BF00BF00BF00BF00BF00BF00BFB6
:1032200000BF00BF00BF00BF00BF00BF00BF00BFA6
:1032300000BF00BF00BF00BF00BF00BF00BF00BF96
:1032400000BF00BF00BF00BF00BF00BF00BF00BF86
:1032500000BF00BF00BF00BF00BF00BF00BF00BF76
:1032600000BF00BF00BF00BF00BF00BF00BF00BF66
:1032700000BF00BFEC630120FFF720FAB000FFF7AA
:103280001DFAAC6300BF00BF00BF00BF00BF00BF9E
:1032900000BF00BF00BF00BF00BF00BF00BF00BF36
:1032A00000BF00BF00BF00BF00BF00BF00BF00BF26
:1032B00000BF00BF00BF00BF00BF00BF00BF00BF16
:1032C00000BF00BF70BD2DE9FE430F46044602A9B2
:1032D000794800F0BCFD794D794EDFF8E88148B1BE
:1032E000822028602220794630608220C8F80010B1
:1032F000BDE8FE839DF80800800701D4FFF7BCFEFF
:1033000002208DF80000200C8DF80100200A8DF8B5
:1033100002008DF803408DF8047000BF00BF00BFAD
:1033200000BF00BF00BF00BF00BF00BF00BF00BFA5
:1033300000BF00BF00BF00BF00BF00BF00BF00BF95
:1033400000BF00BF00BF00BF00BF00BF00BF00BF85
:1033500000BF00BF00BF00BF00BF564F4FF4802426
:10336000FC6305216846FFF7B0F9BC6300BF00BFEE
:1033700000BF00BF00BF00BF00BF00BF00BF00BF55
:1033800000BF00BF00BF00BF00BF00BF00BF00BF45
:1033900000BF00BF00BF00BF00BF00BF00BF00BF35
:1033A00000BF00BF00BF00BF00BF00BF00202860FB
:1033B00079463060C8F800109AE72DE9FC5F3F4D70
:1033C0003F4E404F5FEA020A8B4604464FF000082A
:1033D0000DD001A9384800F03AFD80B18220286064
:1033E00021203060784638608220BDE8FC9FC5F817
:1033F00000807846C6F8008038600020F5E703209A
:103400008DF80000200C8DF80100200A8DF80200D4
:103410008DF8034000BF00BF00BF00BF00BF00BF6A
:1034200000BF00BF00BF00BF00BF00BF00BF00BFA4
:1034300000BF00BF00BF00BF00BF00BF00BF00BF94
:1034400000BF00BF00BF00BF00BF00BF00BF00BF84
:1034500000BF00BF174C4FF48029C4F83C900421F2
:103460006846FFF732F951465846FFF73AF9C4F873
:10347000389000BF00BF00BF00BF00BF00BF00BF4B
:1034800000BF00BF00BF00BF00BF00BF00BF00BF44
:1034900000BF00BF00BF00BF00BF00BF00BF00BF34
:1034A00000BF00BF00BF00BF00BF00BF00BF00BF24
:1034B00000BF9CE700C00920A08601006C0000103E
:1034C00070000010740000102DE9F05FFF4EDFF86F
:1034D0000094DFF800A4150083460F464FF0000863
:1034E0000ED000240AE0395D0BEB0400FFF7EBFE81
:1034F000000602D53068BDE8F09F641CAC42F2D3F0
:10350000C6F800807946C9F800800020CAF800108B
:10351000F1E72DE9FC47044601A9EF4800F097FCCC
:10352000EA4DEB4EDFF8AC9348B1822028602220B0
:10353000794630608220C9F80010BDE8FC879DF80C
:103540000400800701D4FFF797FD20208DF80000CC
:1035500020098DF8010020018DF8020000248DF86B
:10356000034000BF00BF00BF00BF00BF00BF00BFDF
:1035700000BF00BF00BF00BF00BF00BF00BF00BF53
:1035800000BF00BF00BF00BF00BF00BF00BF00BF43
:1035900000BF00BF00BF00BF00BF00BF00BF00BF33
:1035A00000BFDFF838834FF48027C8F83C7004214F
:1035B0006846FFF78AF8C8F8387000BF00BF00BF40
:1035C00000BF00BF00BF00BF00BF00BF00BF00BF03
:1035D00000BF00BF00BF00BF00BF00BF00BF00BFF3
:1035E00000BF00BF00BF00BF00BF00BF00BF00BFE3
:1035F00000BF00BF00BF00BF00BF2C607946346031
:103600000020C9F8001098E72DE9FC478A460446D7
:1036100001A9B14800F01BFCAC4DAD4EDFF8B492EF
:1036200040B1822028602220794630608220C9F88B
:10363000001082E703208DF8000020098DF80100BA
:1036400020018DF8020000248DF8034000BF00BF68
:1036500000BF00BF00BF00BF00BF00BF00BF00BF72
:1036600000BF00BF00BF00BF00BF00BF00BF00BF62
:1036700000BF00BF00BF00BF00BF00BF00BF00BF52
:1036800000BF00BF00BF00BF00BF00BFDFF84C821B
:103690004FF48027C8F83C7004216846FFF715F8FE
:1036A000B9115046FFF71DF8C8F8387000BF00BFC9
:1036B00000BF00BF00BF00BF00BF00BF00BF00BF12
:1036C00000BF00BF00BF00BF00BF00BF00BF00BF02
:1036D00000BF00BF00BF00BF00BF00BF00BF00BFF2
:1036E00000BF00BF00BF00BF00BF00BF2C60794615
:1036F00034600020C9F800101FE72DE9F34F83B0B4
:10370000044601A9744800F0A2FB704D704E714F41
:103710004FF0820818B12120C5F800806CE09DF8B8
:103720000400800701D4FFF7A7FCAD208DF800004E
:1037300020098DF8010020018DF802004FF0000BE8
:103740008DF803B000BF00BF00BF00BF00BF00BFC7
:1037500000BF00BF00BF00BF00BF00BF00BF00BF71
:1037600000BF00BF00BF00BF00BF00BF00BF00BF61
:1037700000BF00BF00BF00BF00BF00BF00BF00BF51
:1037800000BF00BFDFF854914FF4802A5446C9F8B7
:103790003CA004216846FEF798FF02210498FEF73A
:1037A00094FFC9F8384000BF00BF00BF00BF00BF92
:1037B00000BF00BF00BF00BF00BF00BF00BF00BF11
:1037C00000BF00BF00BF00BF00BF00BF00BF00BF01
:1037D00000BF00BF00BF00BF00BF00BF00BF00BFF1
:1037E00000BF00BF00BF022401A93B4800F02FFB2F
:1037F00048B12220C5F800803060784638608220C9
:1038000005B0BDE8F08F00BF00BF00BF00BF00BF24
:1038100000BF00BF00BF00BF00BF00BF00BF00BFB0
:1038200000BF00BF00BF00BF00BF00BF00BF00BFA0
:1038300000BF00BF00BF00BF00BF00BF00BF00BF90
:1038400000BF00BF00BFC9F83CA0AD20FEF736FFA7
:10385000049802212044FEF738FFC9F838A000BFC1
:1038600000BF00BF00BF00BF00BF00BF00BF00BF60
:1038700000BF00BF00BF00BF00BF00BF00BF00BF50
:1038800000BF00BF00BF00BF00BF00BF00BF00BF40
:1038900000BF00BF00BF00BF00BF00BF00BFA41C2F
:1038A000A4B2B4F5805F9FD301A90B4800F0CFFA12
:1038B00000287FF430AFFFF729FCC5F800B0784648
:1038C000C6F800B0386000209AE700006C000010D5
:1038D0007000001074000010A086010000C00920D4
:1038E00070B5FD4DFD4EFE4C2AB1FFF766FD00069A
:1038F00009D5206870BD86202060092028607846A0
:103900003060862070BD00202060286078463060DE
:10391000002070BD2DE9F04F89B0DFF8C483DFF8D7
:10392000B8B35FEA02094FF0000607910FD04FF4D9
:10393000805501462A466846FCF73EFDDDE9004712
:10394000284601F0E7FC5FEA000A0CD016E0862169
:10395000C8F800100921CBF800107946DF48016053
:10396000862009B04DE78221C8F800102221CBF84B
:1039700000107946D94801608220F2E7A9EB0605DC
:10398000C7F58050A84200D20546B5F5805F04D047
:1039900020465146FFF738FE80B92046FFF7B9FDB3
:1039A00060B907982A46811907EB0A0001F008FD63
:1039B0002E4420465146FFF7A0FE28B1504601F0A4
:1039C000D8FCD8F80000CCE70027641C4E45D5D3BE
:1039D000504601F0CEFC0020C8F800007946CBF834
:1039E0000000BE4801600020BBE72DE9FF4F8DB00D
:1039F0000D46DDF868900026B94C07935FEA09018F
:103A00003FD04FF4805701463A466846FCF7D4FC55
:103A1000DDE900B10C913A46691C6846FCF7CCFC24
:103A2000DDE90010CDE904013A4668460F99FCF73C
:103A3000C3FCDDE9008500BFA9EB0607C5F5805092
:103A4000B84200D2074625B1D8457CD10C988542B2
:103A500079D14FF4805001F05DFC5FEA000A1BD081
:103A6000D8454FD10C9885424CD12A464FEA0830B0
:103A70005146FFF7A2FC000618D5504601F079FC2C
:103A800079E08620206094480921016078469349B6
:103A90000860862011B0B4E6822020608E48222182
:103AA000016079468D4801608220F3E705988045E2
:103AB00009D1049901EB0030C1F580525144FFF760
:103AC0007CFC0006D9D44046FFF723FD0006D4D481
:103AD00007983A46811905EB0A0001F071FCEA19D2
:103AE0004FEA08305146FFF7EFFC0006C5D40599B0
:103AF000884533D1049800EB01300499C1F5805218
:103B0000514427E0059988450AD1049800EB01301B
:103B10000499C1F580525146FFF74FFC0006ACD422
:103B20004046FFF7F6FC0006A7D407983A468119ED
:103B30000F983044FFF7C8FC00069ED405998845CD
:103B40000CD1049800E00DE000EB01300499C1F5C0
:103B500080525146FFF7B8FC00068ED4504601F063
:103B600008FC0AE007983A4681190F983044FFF79D
:103B7000ABFC000601D520688CE73E44002508F127
:103B800001084E45FFF458AF5349002020600860FB
:103B900078465249086000207CE72DE9F0474FF055
:103BA000000900BF00BF00BF00BF00BF00BF00BFD3
:103BB00000BF00BF00BF00BF00BF00BF00BF00BF0D
:103BC00000BF00BF00BF00BF00BF00BF00BF00BFFD
:103BD00000BF00BF00BF00BF00BF00BF00BF00BFED
:103BE00000BF404E4FF48025F5639F20FEF766FD31
:103BF0000020FEF763FD00F0FF080020FEF75EFDE9
:103C0000C4B20020FEF75AFDC1B2B56300BF00BFC9
:103C100000BF00BF00BF00BF00BF00BF00BF00BFAC
:103C200000BF00BF00BF00BF00BF00BF00BF00BF9C
:103C300000BF00BF00BF00BF00BF00BF00BF00BF8C
:103C400000BF00BF00BF00BF00BF00BF244D224E19
:103C5000224FB8F1BF0F03D1252C0AD0262C08D053
:103C60008220286021203060784638608220BDE8BC
:103C7000F0871D48412912D04FF48002422912D00A
:103C80004A2910D0C0F800900020FFF789FAC5F843
:103C900000907846C6F8009038600020E7E74FF4BF
:103CA00000110160F0E70260EEE72DE9F84F694688
:103CB0000E4800F0CCF88227094C074D074E4FF014
:103CC000220A002862D19DF80000800701D4FFF786
:103CD000D3F900BF00BF0BE07000001074000010AB
:103CE0006C00001000C0092014010010A086010023
:103CF00000BF00BF00BF00BF00BF00BF00BF00BFCC
:103D000000BF00BF00BF00BF00BF00BF00BF00BFBB
:103D100000BF00BF00BF00BF00BF00BF00BF00BFAB
:103D200000BF00BF00BF00BF00BF00BFDFF8EC91C5
:103D30004FF48028C9F83C806020FEF7BFFCC9F82A
:103D4000388000BF00BF00BF00BF00BF00BF00BF82
:103D500000BF00BF00BF00BF00BF00BF00BF00BF6B
:103D600000BF00BF00BF00BF00BF00BF00BF00BF5B
:103D700000BF00BF00BF00BF00BF00BF00BF00BF4B
:103D800000BF6946664800F062F838B1276078469F
:103D9000C5F800A030608220BDE8F88F00202060C8
:103DA0002860784630600020F6E75E48006870477B
:103DB0004FF4805070472DE9F04FDFF86C81DFF849
:103DC0006CB189B00F0004464FF0000626D04FF4C6
:103DD000805501462A466846FCF7EEFADDE900A167
:103DE00005912A46214606A8FCF7E6FADDE90640D9
:103DF0004FF00009BD1BC0F58051A94200D20D460D
:103E000020B1544515D10599884212D12046FFF7BB
:103E100080FB00060DD5D8F80000A2E58621C8F881
:103E200000100921CBF80010794641480160862036
:103E300097E52E44641C4846BE42DBD3C8F8000018
:103E40007946CBF800003A480160002089E52DE969
:103E5000F041384C0F460646A56806E0A068401BB6
:103E6000B04202D30120BDE8F081384600F003F8EB
:103E70000028F3D1F7E770B5044600BF00BF00BFCC
:103E800000BF00BF00BF00BF00BF00BF00BF00BF3A
:103E900000BF00BF00BF00BF00BF00BF00BF00BF2A
:103EA00000BF00BF00BF00BF00BF00BF00BF00BF1A
:103EB00000BF00BF00BF00BF00BF184E4FF48025F9
:103EC000F5630520FEF7FAFB0020FEF7F7FB2070F4
:103ED000B56300BF00BF00BF00BF00BF00BF00BF91
:103EE00000BF00BF00BF00BF00BF00BF00BF00BFDA
:103EF00000BF00BF00BF00BF00BF00BF00BF00BFCA
:103F000000BF00BF00BF00BF00BF00BF00BF00BFB9
:103F100000BF207800F0010070BD000000C0092043
:103F200020A10700140100106C00001070000010A8
:103F300074000010008000402DE9FF4703A9FE48EF
:103F400000F063FBFD4DFE4EDFF8F89350B1822088
:103F500028602120794630608220C9F8001004B022
:103F6000BDE8F0879DF80C00800701D4FFF784F8C6
:103F700042208DF800000024CDF80140CDF8054026
:103F8000ADF8094000BF00BF00BF00BF00BF00BFC9
:103F900000BF00BF00BF00BF00BF00BF00BF00BF29
:103FA00000BF00BF00BF00BF00BF00BF00BF00BF19
:103FB00000BF00BF00BF00BF00BF00BF00BF00BF09
:103FC00000BF00BFDFF880834FF48027C8F83C7043
:103FD0000B216846FEF779FBC8F8387000BF00BFB8
:103FE00000BF00BF00BF00BF00BF00BF00BF00BFD9
:103FF00000BF00BF00BF00BF00BF00BF00BF00BFC9
:1040000000BF00BF00BF00BF00BF00BF00BF00BFB8
:1040100000BF00BF00BF00BF00BF00BF2C607946DB
:1040200034600020C9F8001099E72DE9F34F85B0FE
:10403000044603A9C04800F0E8FAC04DC04EC14F85
:104040004FF0820B18B12120C5F800B060E0FFF7F7
:1040500013F842208DF800004FF0000ACDF801A0BF
:10406000CDF805A0ADF809A000BF00BF00BF00BF9C
:1040700000BF00BF00BF00BF00BF00BF00BF00BF48
:1040800000BF00BF00BF00BF00BF00BF00BF00BF38
:1040900000BF00BF00BF00BF00BF00BF00BF00BF28
:1040A00000BF00BF00BF00BFDFF89C924FF4802824
:1040B000C9F83C800B216846FEF707FBC9F8388039
:1040C00000BF00BF00BF00BF00BF00BF00BF00BFF8
:1040D00000BF00BF00BF00BF00BF00BF00BF00BFE8
:1040E00000BF00BF00BF00BF00BF00BF00BF00BFD8
:1040F00000BF00BF00BF00BF00BF00BF00BF00BFC8
:1041000003A98D4800F081FA48B12220C5F800B01B
:10411000306078463860822007B0BDE8F08F9DF8A7
:104120000C00800701D4FEF7A7FF02208DF80000E5
:10413000200C8DF80100200A8DF8020006988DF8F9
:1041400003408DF8040000BF00BF00BF00BF00BFE8
:1041500000BF00BF00BF00BF00BF00BF00BF00BF67
:1041600000BF00BF00BF00BF00BF00BF00BF00BF57
:1041700000BF00BF00BF00BF00BF00BF00BF00BF47
:1041800000BF00BF00BF4446C846C9F83C400521F7
:104190006846FEF79AFAC8F8384000BF00BF00BF73
:1041A00000BF00BF00BF00BF00BF00BF00BF00BF17
:1041B00000BF00BF00BF00BF00BF00BF00BF00BF07
:1041C00000BF00BF00BF00BF00BF00BF00BF00BFF7
:1041D00000BF00BF00BF00BF00BFC5F800A0784609
:1041E000C6F800A03860002096E72DE9F05F534E36
:1041F000DFF84C91DFF84CA1150083460F464FF0D5
:1042000000080ED000240AE0395D0BEB0400FFF734
:104210000CFF000602D53068BDE8F09F641CAC427C
:10422000F2D3C6F800807946C9F800800020CAF8A9
:104230000010F1E72DE9F34F0024404D404E414F6F
:10424000C3B080464FF0820A4FF0210BA14641A92E
:10425000394800F0DAF900287CD19DF80401800784
:1042600001D4FEF709FF02208DF800004FEA181074
:104270008DF8010004EB08108DF8020044988DF8C9
:10428000039000EB04214FF4807201A801F098F82C
:1042900000BF00BF00BF00BF00BF00BF00BF00BF26
:1042A00000BF00BF00BF00BF00BF00BF00BF00BF16
:1042B00000BF00BF00BF00BF00BF00BF00BF00BF06
:1042C00000BF00BF00BF00BF00BF00BF00BF00BFF6
:1042D0001D494FF48020C8634FF482716846FEF791
:1042E000F4F919494FF48020886300BF00BF00BF74
:1042F00000BF00BF00BF00BF00BF00BF00BF00BFC6
:1043000000BF00BF00BF00BF00BF00BF00BF00BFB5
:1043100000BF00BF00BF00BF00BF00BF00BF00BFA5
:1043200000BF00BF00BF00BF00BF641CE4B2102C80
:104330008DD341A900480AE0A08601006C0000105E
:10434000700000107400001000C0092002E000F0AE
:104350005CF940B1C5F800A07846C6F800B03860F6
:10436000822045B0D9E6FEF7D1FEC5F80090784628
:10437000C6F8009038600020F3E72DE9F04F89B0CF
:10438000DFF85483DFF854B35FEA02094FF0000608
:1043900007910FD04FF4805501462A466846FCF736
:1043A0000BF8DDE90047284600F0B4FF5FEA000A99
:1043B0000CD016E08621C8F800100921CBF80010B7
:1043C0007946C7480160862009B0A6E68221C8F870
:1043D00000102221CBF800107946C14801608220EC
:1043E000F2E7A9EB0605C7F58050A84200D20546C2
:1043F000B5F5805F04D020465146FFF705F980B936
:104400002046FFF786F860B907982A46811907EB1E
:104410000A0000F0D5FF2E4420465146FFF70AFF60
:1044200028B1504600F0A5FFD8F80000CCE70027DF
:10443000641C4E45D5D3504600F09BFF0020C8F8C1
:1044400000007946CBF80000A54801600020BBE7DA
:104450002DE9FF4F8DB00D46DDF8689000269E4C8B
:1044600007935FEA09013ED04FF4805701463A4670
:104470006846FBF7A1FFDDE900B10C913A46691CE3
:104480006846FBF799FFDDE90010CDE904013A46E3
:1044900068460F99FBF790FFDDE90085A9EB060759
:1044A000C5F58050B84200D2074625B1D8457CD129
:1044B0000C98854279D14FF4805000F02BFF5FEAD1
:1044C000000A1BD0D8454FD10C9885424CD12A46C2
:1044D0004FEA08305146FEF770FF000618D55046E7
:1044E00000F047FF79E0862020607C4809210160C8
:1044F00078467B490860862011B00EE68220206055
:104500007648222101607946754801608220F3E7F0
:104510000598804509D1049901EB0030C1F580521E
:104520005144FEF74AFF0006D9D44046FEF7F1FF9A
:104530000006D4D407983A46811905EB0A0000F02A
:104540003FFFEA194FEA08305146FFF74EFE0006DA
:10455000C5D40599884533D1049800EB01300499FE
:10456000C1F58052514427E0059988450AD1049845
:1045700000EB01300499C1F580525146FEF71DFF52
:104580000006ACD44046FEF7C4FF0006A7D4079847
:104590003A4681190F983044FFF727FE00069ED453
:1045A000059988450CD1049800E00DE000EB01303E
:1045B0000499C1F580525146FFF717FE00068ED4CC
:1045C000504600F0D6FE0AE007983A4681190F9847
:1045D0003044FFF70AFE000601D520688CE73E4410
:1045E000002508F101084E45FFF458AF3B49002073
:1045F0002060086078463A49086000207CE74FF464
:10460000800070474FF4805070472DE9F041354CE1
:104610000F460646A56806E0A068401BB04202D3DC
:104620000120BDE8F081384600F003F80028F3D1FE
:10463000F7E770B5044600BF00BF00BF00BF00BF72
:1046400000BF00BF00BF00BF00BF00BF00BF00BF72
:1046500000BF00BF00BF00BF00BF00BF00BF00BF62
:1046600000BF00BF00BF00BF00BF00BF00BF00BF52
:1046700000BF00BF00BF1C4E4FF48025F56305202E
:10468000FEF71CF80020FEF719F82070B56300BF94
:1046900000BF00BF00BF00BF00BF00BF00BF00BF22
:1046A00000BF00BF00BF00BF00BF00BF00BF00BF12
:1046B00000BF00BF00BF00BF00BF00BF00BF00BF02
:1046C00000BF00BF00BF00BF00BF00BF00BF207819
:1046D00000F0010070BD00006C00001070000010C0
:1046E000740000100080004000C0092070B504462E
:1046F00000BF00BF00BF00BF00BF00BF00BF00BFC2
:1047000000BF00BF00BF00BF00BF00BF00BF00BFB1
:1047100000BF00BF00BF00BF00BF00BF00BF00BFA1
:1047200000BF00BF00BF00BF00BF00BF00BF00BF91
:10473000FF4E4FF08065F563D720FDF7BFFF0020E7
:10474000FDF7BCFF2070B56300BF00BF00BF00BF16
:1047500000BF00BF00BF00BF00BF00BF00BF00BF61
:1047600000BF00BF00BF00BF00BF00BF00BF00BF51
:1047700000BF00BF00BF00BF00BF00BF00BF00BF41
:1047800000BF00BF00BF00BF207800F03D012C2912
:1047900002D04FF0FF3070BD000601D5002070BD83
:1047A000012070BDE34900200860E34908607846B5
:1047B000E2490860002070472DE9FE4FDD4EDE4FD4
:1047C000DFF878835FEA02098A4615D001464FF484
:1047D000047201A8FBF7F0FDDDE90154D84800F0B0
:1047E00025FC90B1822030602120794638608220FB
:1047F000C8F80010BDE8FE8F862030600920794699
:1048000038608620C8F80010F4E7E8208DF8000032
:10481000A8098DF80100A80040EA24208DF80200C4
:104820008DF8034000BF00BF00BF00BF00BF00BF46
:1048300000BF00BF00BF00BF00BF00BF00BF00BF80
:1048400000BF00BF00BF00BF00BF00BF00BF00BF70
:1048500000BF00BF00BF00BF00BF00BF00BF00BF60
:1048600000BF00BFB24D4FF08064EC630421684686
:10487000FDF72BFF04216846FDF733FF49465046FC
:10488000FDF72FFFAC6300BF00BF00BF00BF00BF3C
:1048900000BF00BF00BF00BF00BF00BF00BF00BF20
:1048A00000BF00BF00BF00BF00BF00BF00BF00BF10
:1048B00000BF00BF00BF00BF00BF00BF00BF00BF00
:1048C00000BF00BF00BF0020306079463860C8F8E4
:1048D00000108FE72DE9F04FADF5137D0C46DDF8A4
:1048E00070820026DFF84C92DFF84CA2DFF84CB261
:1048F00015468B935FEA08012AD04FF404770146EE
:104900003A4685A8FBF758FDDDE985018D918A902F
:104910003A46611C85A8FBF74FFDDDE985018891CA
:104920008C903A4629468EA8FBF746FDDDE98E5469
:1049300001A88E90824800F079FBB8B18221222034
:10494000C9F80010CAF800007846CBF8000015E15D
:104950008620C9F8000009207946CAF800008620A0
:10496000CBF800100DF5137DBDE8F08FA8EB06071E
:10497000C4F50470B84200D207462CB18A9885422B
:104980007ED18D9884427BD1FF224FF40571684619
:10499000FBF71CFD87208DF8000000208DF801003A
:1049A0008DF802008DF803008A9885420FD18D980A
:1049B00084420CD105EB45102246000101A9FFF706
:1049C000FBFE8B983A4681198E98204403E08B9821
:1049D0003A46811901A800F0F3FC8C9885420BD16E
:1049E000889900EB401001EB0010C1F504720B46F2
:1049F0008E991944FFF7E0FE00BF00BF00BF00BF63
:104A000000BF00BF00BF00BF00BF00BF00BF00BFAE
:104A100000BF00BF00BF00BF00BF00BF00BF00BF9E
:104A200000BF00BF00BF00BF00BF00BF00BF00BF8E
:104A300000BF00BF00BF00BF3D484FF08061C163B1
:104A40004FF405716846FDF740FE39494FF080602C
:104A5000886300BF00BF00BF00BF00BF00BF00BF32
:104A600000BF00BF00BF00BF00BF00BF00BF00BF4E
:104A700000BF00BF00BF00BF00BF00BF00BF00E01D
:104A80000CE000BF00BF00BF00BF00BF00BF00BF01
:104A900000BF00BF00BF002C72D0CEE055208DF8C3
:104AA0000000A8098DF80100A8008DF80200002080
:104AB0008DF8030000BF00BF00BF00BF00BF00BFF4
:104AC00000BF00BF00BF00BF00BF00BF00BF00BFEE
:104AD00000BF00BF00BF00BF00BF00BF00BF00BFDE
:104AE00000BF00BF00BF00BF00BF00BF00BF00BFCE
:104AF00000BF00BF0E484FF08061C16304216846CB
:104B0000FDF7E3FD0A494FF08060886300BF00BFF6
:104B100000BF00BF00BF00BF00BF00BF00BF00BF9D
:104B200000BF00BF00BF00BF00BF00BF00BF09E063
:104B300000C009206C00001070000010740000100C
:104B4000A086010000BF00BF00BF00BF00BF00BFC4
:104B500000BF00BF00BF00BF00BF00BF00BF00BF5D
:104B600000BFFA4800F062FA58B18221C9F800107B
:104B700022207946CAF80000CBF800108220F1E626
:104B800061E087208DF8000000208DF80100200AE8
:104B90008DF802008DF8034000BF00BF00BF00BFCA
:104BA00000BF00BF00BF00BF00BF00BF00BF00BF0D
:104BB00000BF00BF00BF00BF00BF00BF00BF00BFFD
:104BC00000BF00BF00BF00BF00BF00BF00BF00BFED
:104BD00000BF00BF00BF00BFDD494FF08060C86369
:104BE00004216846FDF771FD8B9839463044FDF786
:104BF0006CFDD7494FF08060886300BF00BF00BFE5
:104C000000BF00BF00BF00BF00BF00BF00BF00BFAC
:104C100000BF00BF00BF00BF00BF00BF00BF00BF9C
:104C200000BF00BF00BF00BF00BF00BF00BF00BF8C
:104C300000BF00BF00BF00BF00BF8A98854204D1FB
:104C40008D98844201D1862000E089208DF80000F3
:104C5000A8098DF80100A8008DF8020000208DF849
:104C6000030000BF00BF00BF00BF00BF00BF00BF08
:104C700000BF00BF00BF00BF00BF00BF00BF00BF3C
:104C800000BF00BF00BF00BF00BF00BF00BF00BF2C
:104C900000BF00BF00BF00BF00BF00BF00BF00BF1C
:104CA00000BFAB484FF08064C46304216846FDF741
:104CB0000CFDA748846300BF00BF00BF00BF00BF5A
:104CC00000BF00BF00BF00BF00BF00BF00BF00BFEC
:104CD00000BF00BF00BF00BF00BF00BF00BF00BFDC
:104CE00000BF00BF00BF00BF00BF00BF00BF00BFCC
:104CF00000BF00BF00BF3E4400246D1C4645FFF4CA
:104D000019AE0020C9F800007946CAF80000CBF8B7
:104D1000001027E62DE9F04FADF5057D00BF00BF7F
:104D200000BF00BF00BF00BF00BF00BF00BF00BF8B
:104D300000BF00BF00BF00BF00BF00BF00BF00BF7B
:104D400000BF00BF00BF00BF00BF00BF00BF00BF6B
:104D500000BF00BF00BF00BF00BF00BFDFF8F09181
:104D60004FF080644D46C9F83C40D720FDF7A6FCC3
:104D70000020FDF7A3FCAC6300BF00BF00BF00BF75
:104D800000BF00BF00BF00BF00BF00BF00BF00BF2B
:104D900000BF00BF00BF00BF00BF00BF00BF00BF1B
:104DA00000BF00BF00BF00BF00BF00BF00BF00BF0B
:104DB00000BF00BF00BF00BF00F03D00654D664E64
:104DC000664F4FF0820B2C2854D100BF00BF00BFAC
:104DD00000BF00BF00BF00BF00BF00BF00BF00BFDB
:104DE00000BF00BF00BF00BF00BF00BF00BF00BFCB
:104DF00000BF00BF00BF00BF00BF00BF00BF00BFBB
:104E000000BF00BF00BF00BF00BFA046CA46C9F830
:104E10003C409F20FDF752FC0020FDF74FFCC4B240
:104E20000020FDF74BFCC0B2C9F8388000BF00BFBE
:104E300000BF00BF00BF00BF00BF00BF00BF00BF7A
:104E400000BF00BF00BF00BF00BF00BF00BF00BF6A
:104E500000BF00BF00BF00BF00BF00BF00BF00BF5A
:104E600000BF00BF00BF00BF00BF00BF1F2C01D1AB
:104E7000262809D02120C5F800B030607846386077
:104E800082200DF5057D6FE54FF4057BFF22594625
:104E90006846FBF79BFA87208DF8000000248DF808
:104EA00001408DF802408DF8034000BF00BF00BFF5
:104EB00000BF00BF00BF00BF00BF00BF00BF00BFFA
:104EC00000BF00BF00BF00BF00BF00BF00BF00BFEA
:104ED00000BF00BF00BF00BF00BF00BF00BF00BFDA
:104EE00000BF00BF00BF00BF00BFC1464046D04664
:104EF000CAF83C0059466846FDF7E7FBC8F8389009
:104F000000BF00BF00BF00BF00BF00BF00BF00BFA9
:104F100000BF00BF00BF00BF00BF00BF00BF00BF99
:104F200000BF00BF00BF00BF00BF00BF00BF00BF89
:104F300000BF00BF00BF00BF00BF00BF00BF00BF79
:104F40002C6078463460386000209AE7A086010023
:104F500000C009206C0000107000001074000010E8
:104F600070B500BF00BF00BF00BF00BF00BF00BFE3
:104F700000BF00BF00BF00BF00BF00BF00BF00BF39
:104F800000BF00BF00BF00BF00BF00BF00BF00BF29
:104F900000BF00BF00BF00BF00BF00BF00BF00BF19
:104FA00000BF2B4D4FF08064EC6304212948FDF7CE
:104FB0008CFBAC6300BF00BF00BF00BF00BF00BFE1
:104FC00000BF00BF00BF00BF00BF00BF00BF00BFE9
:104FD00000BF00BF00BF00BF00BF00BF00BF00BFD9
:104FE00000BF00BF00BF00BF00BF00BF00BF00BFC9
:104FF00000BF00BF184800F019F81849184A194BAB
:1050000038B1822008602220106078461860822023
:1050100070BD00200860106078461860002070BDE8
:105020004FF4041070474FF404707047F8B50E4EFB
:105030000546B46805E0B068001BA84201D3012012
:10504000F8BD6846FFF752FB0028F4D1F8BD000018
:1050500000C00920FC03000000B4C4046C00001070
:1050600070000010740000100080004000207047A5
:105070009D49822008609D492120086078469C490E
:105080000860822070479849822008609749222052
:1050900008607846964908608220704792498220CD
:1050A0000860924922200860784691490860822071
:1050B00070472DE9F041002400BF00BF00BF00BFD2
:1050C00000BF00BF00BF00BF00BF00BF00BF00BFE8
:1050D00000BF00BF00BF00BF00BF00BF00BF00BFD8
:1050E00000BF00BF00BF00BF00BF00BF00BF00BFC8
:1050F00000BF00BF00BF00BF7E4D4FF08066EE6373
:105100003712EF639F20FDF7D9FA0020FDF7D6FA9A
:1051100060F307040020FDF7D1FA60F30F240020AC
:10512000FDF7CCFA60F31744AE63AF6300BF00BF76
:1051300000BF00BF00BF00BF00BF00BF00BF00BF77
:1051400000BF00BF00BF00BF00BF00BF00BF00BF67
:1051500000BF00BF00BF00BF00BF00BF00BF00BF57
:1051600000BF00BF00BF00BF00BF00BF6249601AA0
:105170008C4220D00EDCA4F21F64B4F5005418D089
:105180005E48201817D0B0F5803F14D0B0F5003F2E
:105190000BD110E05A49401805D05A4940180CD09C
:1051A0005949C84201D1022400E000242046BDE84C
:1051B000F0810124FAE70324F8E70424FEF7BCFE9B
:1051C000F4E75248007828B1514900EBC00051F88B
:1051D000200000474449822008604449212008609B
:1051E0007846434908608220704770B5FFF761FF39
:1051F00046493E4D3E4E3C4C087050B1444900EB90
:10520000C00001EB800080688047000609D5206857
:1052100070BD822020602120286078463060822086
:1052200070BD00202060286078463060002070BD8E
:105230002DE9F041354B2D4D2D4E1B782A4C5BB19D
:1052400092B1334F03EBC30307EB83031B6998470A
:10525000000611D52068AAE782202060212028605E
:10526000784630608220A2E78620206009202860EE
:105270007846306086209AE70020206028607846D3
:105280003060002093E7F8B5204C184D184E277871
:10529000154CDDF818C087B1BCF1000F15D0CDF862
:1052A00000C0DFF86CC007EBC7070CEB8707FF698E
:1052B000B847000611D52068F8BD82202060222062
:1052C0002860784630608220F8BD86202060092062
:1052D0002860784630608620F8BD00202060286075
:1052E000784630600020F8BD6C000010700000109F
:1052F0007400001000C00920C22018005D05ECFFFA
:1053000003FBD6FF00FFFEFF0001F8FF18010010AD
:10531000245D000070B50646FBF760F8056806F1ED
:105320000B0020F00704B4429CBF002070BD2B4648
:105330006A68BAB11068A04210D304F1080188422B
:105340003CBF5068586007D351681019416011681C
:10535000091B016058601460101D70BD134652682F
:10536000002AE7D12146284600F0C5F80028DED102
:1053700070BD70B50446051FFBF730F80068002CBF
:1053800014BF446870BD002C18BFAC423CBF20461F
:105390006468F8D301680A18AA4218BF456003D1AF
:1053A0002A6805461144016028684119A1421CBFC2
:1053B0006C6070BD6168696021680844286070BDD8
:1053C000032A40F2308010F0030C00F0158011F831
:1053D000013BBCF1020F624498BF11F801CB00F809
:1053E000013B38BF11F8013BA2F1040298BF00F85D
:1053F00001CB38BF00F8013B11F0030300F025801A
:10540000083AC0F0088051F8043B083A51F804CB40
:10541000A0E80810F5E7121D5CBF51F8043B40F806
:10542000043BAFF30080D20724BF11F8013B11F811
:1054300001CB48BF11F8012B24BF00F8013B00F855
:1054400001CB48BF00F8012B704710B5203AC0F0DF
:105450000B80B1E81850203AA0E81850B1E8185075
:10546000A0E81850BFF4F5AF5FEA027C24BFB1E8B2
:105470001850A0E8185044BF18C918C0BDE8104023
:105480005FEA827C24BF51F8043B40F8043B08BF2C
:105490007047D20728BF31F8023B48BF11F8012BF3
:1054A00028BF20F8023B48BF00F8012B70474FF09F
:1054B00000020429C0F0128010F0030C00F060809C
:1054C000CCF1040CBCF1020F18BF00F8012BA8BFEF
:1054D00020F8022BA1EB0C0100F052B85FEAC17C6E
:1054E00024BF00F8012B00F8012B48BF00F8012B66
:1054F00070477047704738B504460A460020694631
:10550000AFF30080002808BF38BD0246009920464E
:1055100000F05BF8012038BD012000F070B8F8B54C
:10552000AFF30080054600200C46102000BF064661
:10553000A819A0420DD9324669460020AFF3008079
:10554000070008BF00F05BF80098A04218BF0546AE
:10555000C419FAF743FF05600746F01D20F0070065
:1055600046192846FAF73EFFB44208BFF8BDA21B11
:1055700031463868BDE8F84000F027B84FF0000227
:1055800000B5134694469646203922BFA0E80C5039
:10559000A0E80C50B1F12001BFF4F7AF090728BF14
:1055A000A0E80C5048BF0CC05DF804EB890028BF90
:1055B00040F8042B08BF704748BF20F8022B11F0B9
:1055C000804F18BF00F8012B7047034640688C4697
:1055D000002818BF88423CBF03464068F8D31868CB
:1055E0001844884207D00CF1030020F00700001D8A
:1055F000411A521A0146081D0A60FFF7BABE10B5DB
:1056000000F038F8BDE8104000F02EB87546FAF703
:10561000F1FEAE4605006946534620F00700854678
:1056200018B020B5FAF7CAFDBDE820404FF00006DB
:105630004FF000074FF000084FF0000B21F007017A
:10564000AC46ACE8C009ACE8C009ACE8C009ACE8BD
:10565000C0098D46704710B50446AFF30080204660
:10566000BDE81040FAF77DBD002801D000F02AB84F
:105670007047000010B5012805D0002103A000F0FC
:1056800027F8012010BD09A1F8E70000534947524F
:10569000544D454D3A204F7574206F662068656102
:1056A00070206D656D6F7279000000003A204865CA
:1056B0006170206D656D6F727920636F72727570A5
:1056C0007465640001491820ABBEFEE726000200A5
:1056D00070B505460C460A2000E06D1C00F011F87C
:1056E00035B128780028F8D102E0641C00F009F8F0
:1056F00014B120780028F8D1BDE870400A20AFF33B
:10570000008008B569468DF800000320ABBE08BDD7
:1057100000050F0A1B1E141133363C39282D272291
:1057200063666C69787D777250555F5A4B4E444181
:10573000C3C6CCC9D8DDD7D2F0F5FFFAEBEEE4E171
:10574000A0A5AFAABBBEB4B193969C99888D878261
:1057500083868C89989D9792B0B5BFBAABAEA4A151
:10576000E0E5EFEAFBFEF4F1D3D6DCD9C8CDC7C241
:1057700040454F4A5B5E545173767C79686D676231
:1057800023262C29383D373210151F1A0B0E040121
:1057900003060C09181D171230353F3A2B2E242111
:1057A00060656F6A7B7E747153565C59484D474201
:1057B000C0C5CFCADBDED4D1F3F6FCF9E8EDE7E2F1
:1057C000A3A6ACA9B8BDB7B290959F9A8B8E8481E1
:1057D00080858F8A9B9E9491B3B6BCB9A8ADA7A2D1
:1057E000E3E6ECE9F8FDF7F2D0D5DFDACBCEC4C1C1
:1057F00043464C49585D575270757F7A6B6E6461B1
:1058000020252F2A3B3E343113161C19080D0702A0
:1058100000002110422063308440A550C660E7702C
:10582000088129914AA16BB18CC1ADD1CEE1EFF1D4
:105830003112100273325222B5529442F772D6627C
:10584000399318837BB35AA3BDD39CC3FFF3DEE324
:105850006224433420040114E664C774A4448554CC
:105860006AA54BB528850995EEE5CFF5ACC58DD574
:105870005336722611163006D776F6669556B4461C
:105880005BB77AA719973887DFF7FEE79DD7BCC7C4
:10589000C448E5588668A77840086118022823386C
:1058A000CCC9EDD98EE9AFF9488969990AA92BB914
:1058B000F55AD44AB77A966A711A500A333A122ABC
:1058C000FDDBDCCBBFFB9EEB799B588B3BBB1AAB64
:1058D000A66C877CE44CC55C222C033C600C411C0C
:1058E000AEED8FFDECCDCDDD2AAD0BBD688D499DB4
:1058F000977EB66ED55EF44E133E322E511E700E5C
:105900009FFFBEEFDDDFFCCF1BBF3AAF599F788F03
:105910008891A981CAB1EBA10CD12DC14EF16FE1E3
:105920008010A100C230E32004502540467067601B
:10593000B9839893FBA3DAB33DC31CD37FE35EF333
:10594000B1029012F322D23235421452776256726B
:10595000EAB5CBA5A89589856EF54FE52CD50DC583
:10596000E234C324A01481046674476424540544BB
:10597000DBA7FAB79987B8975FE77EF71DC73CD7D3
:10598000D326F2369106B01657667676154634560B
:105990004CD96DC90EF92FE9C899E9898AB9ABA923
:1059A0004458654806782768C018E1088238A3285B
:1059B0007DCB5CDB3FEB1EFBF98BD89BBBAB9ABB73
:1059C000754A545A376A167AF10AD01AB32A923AAB
:1059D0002EFD0FED6CDD4DCDAABD8BADE89DC98DC3
:1059E000267C076C645C454CA23C832CE01CC10CFB
:1059F0001FEF3EFF5DCF7CDF9BAFBABFD98FF89F13
:105A0000176E367E554E745E932EB23ED10EF01E4A
:105A1000005EBCE2613FDD83C29C7E20A3FD1F418E
:105A20009DC3217FFCA2401E5F01E3BD3E6082DC7E
:105A3000237D9FC1421CFEA0E1BF5D0380DE3C626E
:105A4000BEE0025CDF81633D7C22C09E1D43A1FF5E
:105A50004618FAA427799BC584DA3866E5BB59074E
:105A6000DB856739BAE406581947A5FB7826C49A3E
:105A7000653BD987045AB8E6A7F91B45C6987A242E
:105A8000F8A6441A99C7257B3A6486D85B05E7B91E
:105A90008CD2306EEDB3510F4E10F2AC2F7193CD0E
:105AA000114FADF3702ECC92D38D6F31B2EC0E50FE
:105AB000AFF1134DCE90722C6D33D18F0C52B0EEEE
:105AC000326C8ED0530DEFB1F0AE4C1291CF2D73DE
:105AD000CA947628ABF517490856B4EA6937D58BCE
:105AE0005709EBB536688AD495CB2977F4AA4816BE
:105AF000E9B7550B88D6346A2B7597C94A14F6A8AE
:105B0000742AC896154BA9F7B6E80A54D7896B359D
:105B1000EB3C904D53444F53352E300002020100B0
:105B20000110000004F80C0001000100000000005A
:105B300000000000000029EFBEADDE41544F4C20B4
:105B4000465072696E744641543132202020000064
:105B500000000000001000000020000000300000E5
:105B600000400000005000000060000000700000D5
:105B7000008000000090000000A0000000B00000C5
:105B800000C0000000D0000000E0000000F00000B5
:105B900000000100008001000000020000800200FF
:105BA00000000300008003000000040000800400E7
:105BB00000000500008005000000060000800600CF
:105BC0000000070000800700FF0F0000FF1F00001B
:105BD000FF2F0000FF3F0000FF4F0000FF5F0000AD
:105BE000FF6F0000FF7F0000FF8F0000FF9F00009D
:105BF000FFAF0000FFBF0000FFCF0000FFDF00008D
:105C0000FFEF0000FFFF0000FF7F0100FFFF01002A
:105C1000FF7F0200FFFF0200FF7F0300FFFF030082
:105C2000FF7F0400FFFF0400FF7F0500FFFF05006A
:105C3000FF7F0600FFFF0600FF7F0700FFFF070052
:105C4000120110010000004051C2031300010420A2
:105C5000480109022000010100803209040000020D
:105C60000806506207058202400000070502024054
:105C7000000000040309041C03410054004F004CC1
:105C80000020002000200020002000200020002014
:105C9000002000280346005000720069006E007466
:105CA00000200046006C00610073006800200020A6
:105CB00000200020002000200020001A0346006978
:105CC0000072006D007700610072006500300030E6
:105CD00000300030000E034D0065006D006F007253
:105CE00000790000AD2100000000000093030000D7
:105CF00000000000000000000000000000000000A4
:105D00000000000000000000000000000000000093
:105D10000000000000000000000000000000000083
:105D2000000000006D5000006D5000007150000038
:105D3000875000007150000087500000875000001D
:105D4000875000009D5000002150000027500000A7
:105D5000154D0000614F0000B9470000A547000045
:105D6000A5470000D54800009D500000AB3D000055
:105D7000B13D00009B3B0000AB3C0000E13800005F
:105D800015390000C9340000EB390000B73D0000B0
:105D9000E32E0000E92E0000E5290000AB3C0000E6
:105DA000E13800003F2C0000EB410000332D0000E3
:105DB000EF2E0000FF450000054600009B3B000061
:105DC000AB3C0000E13800007B430000EB410000E9
:105DD00051440000B73D000000000000000000003A
:105DE00000000000000000000000000000000000B3
:105DF0000000000000000000000000001C5E000029
:105E0000000000101C01000008010000385F0000C5
:105E10001C0100109C6C00002401000041544F4CF8
:105E200020465072696E74280000000000000000D7
:105E30000000D4284B3D00000000000000000000DE
:105E40000000000000000000000000000000000052
:105E50000000000000000000000000000000000042
:105E60000000000000000000000000000000000032
:105E70000000000000000000000000000000001012
:105E80000000000000000000000000000000000012
:105E90000000000000000000000000000000000002
:105EA00000000000000000000000000000000000F2
:105EB00000000000000000000000000000000000E2
:105EC00000000000000000000000000000000000D2
:105ED00000000000000000000000000000000000C2
:105EE00000000000000000000000000000000000B2
:105EF0000000000000093D0000000000000000005C
:105F00000000000000000000000000000000000091
:105F10000000000000000000000000000000000081
:105F20000000000000000000000000000000000071
:105F30000000000000000000756690E962F40ED3D6
:105F4000148AB79256BCD26267D1D520EDC6849B25
:105F500087B7B432AA28C36AD76BD7D62B7A9723D0
:105F6000FA50178704B4F945A04E40B9B848888163
:105F7000CDBC885B95E712116AC7F11965CB832305
:105F8000656E0E3D27BADBF7F4235E9346739B5193
:105F900098C34833C2C3139547775D73B8F9A28A93
:105FA00015B2EAE6904E32A78D83535975D8E9456C
:105FB000F76563250F6A15EFE08D7EA44F4C60A551
:105FC000CE403E4DCDB9826B85F52F08C2762F9617
:105FD0002D2035865D82A6E4648C357402BB3B8A35
:105FE00064AD27AF59D85BAB7A09055207FA3D3F3C
:105FF00050380D0359D8B8D62636C34436C24CFBA8
:00000001FF
